:10000000CE29FF3FFF3FFF3F03138312CF03CF03F0
:100010004F08003C03181128CF0300000000000027
:10002000082800000000000008000313831222309B
:10003000DC00D801D901DA01DB01DC0303194B280C
:100040000310DB0CDA0CD90CD80CD30CD20CD10C6D
:10005000D00C031C1D28DC0303193D285408D807C5
:1000600055080318550FD90756080318560FDA0715
:1000700057080318570FDB0721285408D8075508DD
:100080000318550FD90756080318560FDA075708F3
:100090000318570FDB070800073003138312DA0039
:1000A000DA0B50280800031383124908A0008417B4
:1000B0000130D2004A08D1005208D000510803197B
:1000C0006528D00D5010FF3F5F28D00950088005EB
:1000D0004A08A100080003138312C90CC9132008A1
:1000E00084000130CC00CD014D084B02031D7A285D
:1000F0004C084A02031CAD280130D2002108D1006F
:100100005208D000510803198928D00D5010FF3F24
:100110008328500880044908CF0004200130D20011
:100120002108D1005208D000510803199B28D00D96
:100130005010FF3F9528D009500880054908CF008E
:1001400004204D084B06031DA7284A084C06031936
:10015000AD28CC0A0319CD0A74280800E83003132F
:100160008312CB000330CC00CD01CE014908D00072
:100170004A08D100D201D301E830D4000330D500C1
:100180000030D6000030D70015205008CB005108B1
:10019000CC005208CD005308CE0000305302031D9E
:1001A000DB2800305202031DDB2802305102031D00
:1001B000DB28A33050020318DE283529A330D000F5
:1001C0000230D100D201D3014B08D4004C08D50035
:1001D0004D08D6004E08D7005008D4025108031C21
:1001E000510FD5025208031C520FD6025308031CAC
:1001F000530FD7025408CB005508CC005608CD0049
:100200005708CE000530D0005408CB005508CC006C
:100210005608CD005708CE00500803191629CE0CF9
:10022000CD0CCC0CCB0CCE13FF3F0D29FF304B0572
:10023000D8004C08D0005008D8044D08D0004E0813
:10024000D1005008D8044E08D00050085804D400FB
:100250005408003A031935290130CB02031CCC02A3
:10026000031CCD02031CCE0216290800F030031334
:1002700083129F05F03083169F0483129F1749084D
:10028000D000D00D5010D00D501050089F041F14F6
:100290004C209F1400309F180130D2005208013AC0
:1002A000031D542900004A291E08D200D301520818
:1002B000D300D2015208CA005308CB0083161E088F
:1002C0005204CA005308CB000030CB0483121F1025
:1002D0004A08D0004B08D100080003138312DB0149
:1002E000DA01D9018030D800D10CD00C031C81294F
:1002F0005408D90755080318550FDA070318DB0A05
:100300000310D01F89295408DA0755080318550F20
:10031000DB07DB0CDA0CD90CD80C031C74295B0846
:10032000D3005A08D2005908D1005808D00008005C
:1003300003138312D801D9011030DC00510DD80D00
:10034000D90D5408D8025508031C550FD9020318BB
:10035000B0295408D80755080318550FD9070310BA
:10036000D00DD10DDC0B9E29080003138312500819
:10037000D100D0010830DC005108D40C0318C42986
:10038000DC0BBD29D10100340310C929D40C03189A
:10039000D107D10CD00CDC0BC629080007300313A1
:1003A0008312990018308316850018309F008D3015
:1003B00083129F000530C9000530CA005320A201F6
:1003C0006430A300A4013230A5000030A6002C3018
:1003D000A7000130A800BC30A9000230AA00AB0180
:1003E0002B08043C031C192A013085005030C90039
:1003F0002308CA002408CB006B20023085002308A4
:10040000C9002408CA00AE20043085005030C9005D
:100410002308CA002408CB006B2085012308C900EB
:100420002408CA00AE202B08043A0319192AAB0A83
:10043000F0290330C90036215008AC005108AD0046
:10044000A201003085190130D2005208003A031D84
:100450002A2A682A02302D02031D302A9E302C02DF
:100460000318502A850105140130AB002B08053C08
:10047000031C4F2A013085005030C9002508CA00EE
:100480002608CB006B2085012508C9002608CA0074
:10049000AE202B08053A03194F2AAB0A362A192A2F
:1004A00003302D02031D562A02302C0203185C2A49
:1004B000850104308500192A03302D02031D622AAC
:1004C00002302C02031C682A850102308500192A9B
:1004D0002C08D0002D08D1006430D400D5016D2146
:1004E0000630D4005008C5005108C600540803194E
:1004F0007E2AC60CC50CC613FF3F772A4508AE00FE
:100500004608AF002C08D0002D08D1000A30D400D6
:10051000D5016D210630D4005008BD005108BE0041
:1005200054080319982ABE0CBD0CBE13FF3F912A34
:100530003D08B0003E08B1006430D400D5013D084C
:10054000D0003E08D10098215008B2000030D10000
:100550006430D400D5016D215008C3005108C40097
:100560004308B6004408B7004308BD02031CBE039D
:100570004408BE020A30D400D5013D08D0003E0830
:10058000D10098215008B3000030D1000A30D400C7
:10059000D5016D215008C1005108C2004108B800C2
:1005A0004208B90041083D02D0004208031C013F47
:1005B0003E02D1005008B4000A30D400B5215008E2
:1005C000BF003F08BA004308D0004408D1000A30F9
:1005D000D400D5016D2150084502BD005108031C0F
:1005E000013F4602BE004108D0004208D1000A3057
:1005F000D400D5016D2150083D02D0005108031CE4
:10060000013F3E02D1003F08D002031CD103500835
:10061000B500AB012B08033C031CB42B3230D000D7
:100620002B08500784000008D2005208003A031D2E
:100630001C2B3F30BB005B2B5208013A031D232BC0
:100640002F30BB005B2B5208023A031D2A2B2730A8
:10065000BB005B2B5208033A031D312B2330BB0038
:100660005B2B5208043A031D382B2130BB005B2B57
:100670005208053A031D3F2B2030BB005B2B52086C
:10068000063A031D462B3030BB005B2B5208073A5D
:10069000031D4D2B3830BB005B2B5208083A031D5D
:1006A000542B3C30BB005B2B5208093A031D5B2BDB
:1006B0003E30BB005B2BBC013C08073C031C842B79
:1006C0002208013A031D652B6B2B80303B02031C73
:1006D0006A2B8B2B712B80303B02031C702B9E2BC3
:1006E0008E2B0130D4003B08D000540803197C2B1A
:1006F000D00D5010FF3F762B5008BB003C08073A46
:100700000319842BBC0A5C2BA2012908C9002A0802
:10071000CA00AE20AE2B0130A200712B0230850042
:100720005030C9002308CA002408CB006B20850183
:100730002308C9002408CA00AE20712B02308500AE
:100740005030C9002708CA002808CB006B2085015B
:100750002308C9002408CA00AE20712B2B08033AD5
:100760000319B42BAB0A0A2B192AB52BFF3FFF3F05
:02400E00D43F9D
:00000001FF
